:020000040000FA
:020000002528B1
:080008008F00030803138312AB
:100010008E0004088C000A088D008A010B19112833
:100020001C280B11063081008B018B168B171308CF
:10003000031D930340201C280D088A000C0884002F
:100040000E0883008F0E0F0E09005F205B206430C6
:100050007320262882073F3406345B344F346634DD
:100060006D347D3407347F34673477347C345834CE
:100070005E34793471348207013402340434083434
:10008000F03085058601120884000310840C1030BE
:100090008407000894001218940E14080F392A20BF
:1000A000860012083B2085041208031D59280430DD
:1000B000920092030800900F0800910A08008B013B
:1000C0008B1683168501860181010130810483121C
:1000D000900191010630810003309200F0308505D7
:1000E00086018B17080093001308031D742808006D
:084000000100020003000400AE
:02400E00F13F80
:1042000043006F0070007900720069006700680069
:104210007400200032003000300032002C002000FA
:10422000540075006E006400720061005700610068
:1042300072006500200049006E0063002E0020001F
:10424000200041006C006C002000520069006700F3
:104250006800740073002000520065007300650060
:0A42600072007600650064002E0075
:00000001FF
